:1000000057EF00F0FF00FF002B002B002B002B0010
:100010002B002B002B002B002B002B002B002B0088
:100020002B002B002B002B002B002B002B002B0078
:100030002B002B002B002B002B002B002B0001038F
:100040002B002B002B002B002B002B002B002B0058
:100050002B002B002B002B002B002B002B002B0048
:100060002B002B002B002B002B002B002B002B0038
:100070002B002B002B002B002B002B002B002B0028
:100080002B002B002B002B002B002B002B002B0018
:100090002B002B002B002B002B002B002B002B0008
:1000A0002B002B002B002B002B002B00FF00C2EF9E
:1000B00009F0600E3901D96F000EDB6F000EDD6FA5
:1000C000080EDF6F000EDE6F290E0001F96F960E2D
:1000D000F86F7F0EE82EFED7F82FFCD7F92FFAD74E
:1000E000900E3C01E56F030EE66F000E466E810E2A
:1000F000456E000E486E000E476E0AD0000E472473
:10010000D96E010E4820DA6E000EDF6E474A482A8B
:100110004550475C46504858D8A0F0D7000E486E6E
:10012000000E476EA80E4724D96E000E4820DA6EE6
:10013000000EDF6E474A482A485004E14F0E475CE4
:10014000D8A0F0D7000E486E000E476E000E472470
:10015000D96E020E4820DA6E000EDF6E474A482A3A
:10016000485004E17F0E475CD8A0F0D7000E000194
:100170009A6F020E9B6F05EC08F0000E3E01BC6FFB
:10018000000EBD6F25EC0AF078EC09F03D01F28914
:1001900039019397000E3D01F96F000EFA6FBC9A7A
:1001A00017D03D01F9AB04D0F99B6F00A0F757F0D1
:1001B000F9B76F00A0F757F06F00A0F754F0150ED5
:1001C0000001F86FC60EE82EFED7F82FFCD700F01E
:1001D0003901A3B7E6D7BC8A000E00019A6F020E60
:1001E0009B6F60006BF2D9FF60006FF2DAFF000EC8
:1001F000DF6EC5EC0AF0000E00018F6F000E8E6FEF
:10020000000E8B6F000E8A6F000E896F0A0E886FCA
:10021000000E856F000E846F000E516EC5EC0AF063
:10022000040E056E210E066E43EC0AF0010E4E6EB2
:10023000000E00018F6F000E8E6F000E9A6F020E7F
:100240009B6F60006BF2D9FF60006FF2DAFF000E67
:10025000DF6EC5EC0AF025EC0AF0B290A09E3901E1
:10026000A191DC0E056E210E066E43EC0AF0000E25
:100270003901906F000E916F000E926F93879491E9
:1002800097919191D28CD28EC5EC0AF0B7EC0AF01E
:1002900091EC0AF0000E466E800E456E800E7C6E6C
:1002A000000E7D6EC5EC0AF0AC9EBC8A000E8DD3AC
:1002B000BC8AA2D3C5EC0AF03C0E056E210E066E78
:1002C00043EC0AF0000E376E000E386E000E396EE9
:1002D000000E3A6E000E3B6E000E3C6E000E3D6E40
:1002E000000E3E6EC3EC07F0520E0001F96F2B0EAC
:1002F000F86F000EE82EFED7F82FFCD7F92FFAD7AB
:1003000000F0C60E056E200E066E43EC0AF0A80E35
:10031000056E000E066E8F0E076E220E086E21EC23
:1003200009F0000E0001A76F000EA66F1CD0BAB82E
:1003300003D0F86BF82B02D00001F86BF83BBA50F1
:10034000F819EF0BF819BA6E110E0001F96F3C0E97
:10035000F86FCB0EE82EFED7F82FFCD7F92FFAD77F
:100360000001A64BA72BA75104E1080EA65DD8A05B
:10037000DED7BA88000E2F6E000E306E000E316E82
:10038000000E326E32503110301013E1800E2F5CAF
:10039000D8B00FD0000E2F24D96E010E3020DA6EA7
:1003A000340EDF6E010E2F26000E30223122322253
:1003B000E9D7000E2F6E280E306E000E316E000E43
:1003C000326E325023E1020E315CD8B01FD02FC004
:1003D00005F030C006F031C007F032C008F05FEC25
:1003E0000AF02FC009F030C00AF031C00BF032C063
:1003F0000CF0000E0D6E010E0E6EE2EC06F0800E9B
:100400002F26000E302231223222DBD7000E0001CF
:10041000A76F000EA66F1CD0BAB803D0F86BF82BEC
:1004200002D00001F86BF83BBA50F819EF0BF8193D
:10043000BA6E110E0001F96F3C0EF86FCB0EE82E6C
:10044000FED7F82FFCD7F92FFAD70001A64BA72B20
:10045000A75104E1080EA65DD8A0DED7A80E056E50
:10046000000E066E9EEC09F0FFD7D20E056E220E2E
:10047000066E43EC0AF0A80E056E000E066E000E26
:10048000076E010E086E000E0A6E400E096E88ECB3
:1004900008F0A80E056E000E066E9EEC09F0C5EC85
:1004A0000AF0A80E056E000E066EFA0E076E220EFA
:1004B000086E21EC09F0000E116E010E126EA80EEE
:1004C000136E000E146E3AEC07F011C043F012C028
:1004D00044F043504410D8B4E9D6BD0E056E220E48
:1004E000066E43EC0AF0580E416E000E426E20EE8E
:1004F00007F04350D9264450DA2210EE03F0415061
:10050000E1264250E2226F007FFFE7FF20EE06F077
:100510004350D9264450DA2210EE02F04150E12631
:100520004250E2226F007FFFE7FF20EE05F04350CC
:10053000D9264450DA2210EE01F04150E126425013
:10054000E2226F007FFFE7FF600007F1D9FF600044
:100550000BF1DAFF000EDF6E080E5824586E000E05
:100560005920596E000E5A205A6E000E5B205B6EA9
:10057000A80E1B6E000E1C6EFD0E1D6E210E1E6E53
:1005800058C01FF059C020F05AC021F05BC022F0C3
:1005900017EC05F0A80E056E000E066E9EEC09F035
:1005A000A80E056E000E066EF10E076E220E086E86
:1005B00021EC09F0080E116E010E126EA80E136EDA
:1005C000000E146E3AEC07F011C043F012C044F074
:1005D00043504410D8B402D0020EF7D1000E4D6E35
:1005E000000E3B6E000E3C6E000E3D6E000E3E6E29
:1005F0001E0E056E220E066E43EC0AF013D2C5ECF9
:100600000AF0280E436E010E446E580E416E000E25
:10061000426E20EE03F04350D9264450DA2210EE09
:1006200003F04150E1264250E2226F007FFFE7FFD6
:1006300020EE02F04350D9264450DA2210EE02F0A8
:100640004150E1264250E2226F007FFFE7FF20EE9B
:1006500001F04350D9264450DA2210EE01F0415007
:10066000E1264250E2226F007FFFE7FF600007F1C2
:10067000D9FF60000BF1DAFF000EDF6EA80E1B6ED3
:10068000000E1C6E950E1D6E210E1E6E58C01FF0C2
:1006900059C020F05AC021F05BC022F017EC05F0E1
:1006A000A80E056E000E066E9EEC09F058C0F8F01C
:1006B00059C0F9F05AC0FAF05BC0FBF0080E06D042
:1006C0000001D890FB33FA33F933F833E82EF8D72A
:1006D000F8C07EF0F9C07FF07EC011F07FC012F04C
:1006E000A80E136E000E146E79EC06F0A80E056EBF
:1006F000000E066E9EEC09F0C5EC0AF0400E3B6E53
:10070000000E3C6E000E3D6E000E3E6E000E376E0B
:10071000000E386E000E396E000E3A6E030E55D183
:10072000760E056E220E066E43EC0AF0000E0001F6
:100730007D6F000E7C6F000E336E000E346E000E67
:10074000356E000E366E400E3B6E000E3C6E000E97
:100750003D6E000E3E6E000E376E000E386E000EBF
:10076000396E000E3A6EA70E056E220E066E43EC31
:100770000AF099D0C3EC07F0030E0001F96F080EE0
:10078000F86F770EE82EFED7F82FFCD7F92FFAD79F
:100790005104D8A470D000017C4B7D2B000E332473
:1007A0002F6E280E3420306E000E3520316E000E74
:1007B0003620326E000E436E010E446E2FC005F0DF
:1007C00030C006F031C007F032C008F05FEC0AF02C
:1007D0002FC009F030C00AF031C00BF032C00CF06D
:1007E00043C00DF044C00EF0E2EC06F0456E466AE0
:1007F00045BE46067CC011F07DC012F0A80E136EF7
:10080000000E146E79EC06F0200ED2EC0AF0A80E61
:10081000056E000E066E9EEC09F0200ED2EC0AF07A
:100820002FC007F030C008F031C009F032C00AF024
:10083000F1EC08F0C5EC0AF045504610D8B41BD0D6
:10084000BAB804D00001F86BF82B02D00001F86BA5
:10085000F83BBA50F819EF0BF819BA6E110E0001F7
:10086000F96F3C0EF86FCB0EE82EFED7F82FFCD7B1
:10087000F92FFAD7E5D7800E3324336E000E3420DB
:10088000346E000E3520356E000E3620366E800E2A
:100890003B243B6E000E3C203C6E000E3D203D6E26
:1008A000000E3E203E6E5850335C595034585A501A
:1008B00035585B503658D8B009D0325007E12F2850
:1008C000FF0E3058010E3158D8A054D7BC8A000E04
:1008D000516EC5EC0AF0BA883D0E056E220E066E0A
:1008E00043EC0AF0040E71D0D29CD29EE50E056E48
:1008F000220E066E43EC0AF06D0E056E210E066E9A
:1009000043EC0AF0000E58242F6E280E5920306E4A
:10091000000E5A20316E000E5B20326E000E7D6E8E
:10092000AC8E32503AE12F28FF0E3058010E31586C
:10093000D8B033D07E8EAC8E000E336E280E346E5F
:10094000000E356E000E366E1DD0BA86B40EAB6E3C
:10095000000E7D6E33C005F034C006F035C007F0E0
:1009600036C008F0A6EC0AF07C6EC20E00D000D0B3
:10097000E82EFCD700D0BA96010E3326000E3422A2
:10098000352236222F50335C305034583150355890
:1009900032503658D8B007D0D8D75B0E056E220E2D
:1009A000066E43EC0AF0A30E0001F96F570EF86FC4
:1009B000020EE82EFED7F82FFCD7F92FFAD700F059
:1009C00091D7D29E7E9EAC9E060E4D6E2BD0BB0E56
:1009D000056E210E066E43EC0AF0A30E0001F96FBE
:1009E000570EF86F020EE82EFED7F82FFCD7F92F1E
:1009F000FAD700F0FF0016D04D50000AD8B45AD4F0
:100A0000010AD8B432D5030AD8B4F9D5010AD8B44A
:100A100087D6070AD8B468D7010AD8B4D2D7030A50
:100A2000D8B4D5D7050E4D6443D457EF00F01F0E50
:100A30002C6E000E2D6ECED0250E2E18D8B40CD0F4
:100A400060006FF0D9FF600073F0DAFF6000BBF068
:100A5000DFFF1B4A1C2ABED0000E256E05D025885C
:100A600003D0C00E251217D0600077F0F6FF6000AB
:100A70007BF0F7FF1D4A1E2A08006F00D4FF2EF0FE
:100A80002E50000AD8B4B5D06C0AD8B4E8D7190AE9
:100A9000D8B4E7D79FD025A814D06000B3F0D9FF11
:100AA0006000B7F0DAFF6F0078FF28F06F0078FF82
:100AB00029F06F0078FF2AF06F0078FF2BF0040E0A
:100AC00013D06000B3F0D9FF6000B7F0DAFF6F0019
:100AD00078FF23F06F0074FF24F023C028F024C0B7
:100AE00029F02A6A2B6A020E2C26000E2D22010EF6
:100AF0002E6E2E50040D8B0EF324F66E200EF42075
:100B0000F76E0900F550285C0900F55029580900D6
:100B1000F5502A580900F5502B58D8A005D02E2A98
:100B20000A0E2E18D8A4E5D72EC026F0276A4AD080
:100B300026C023F027C024F0D89023362436D8903E
:100B4000233624368B0E2324F66E200E2420F76ED7
:100B500009006F00D4FF09F009006F00D4FF0AF00C
:100B600009006F00D4FF0BF00A006F00D4FF0CF0F7
:100B700028C005F029C006F02AC007F02BC008F0F5
:100B800047EC08F005C012F006C013F007C014F0DF
:100B900008C015F00A0E166E000E176E000E186EC5
:100BA000000E196EBEEC08F01250300F2E6E600071
:100BB0006FF0D9FF600073F0DAFF6000BBF0DFFF79
:100BC0001B4A1C2A2606D8A027062628B1E127287A
:100BD000D8A4AED7600077F0F6FF60007BF0F7FF97
:100BE0001D4A1E2A08006F00D4FF2EF02E50D8A4F4
:100BF00023D760006FF0D9FF600073F0DAFF000EBA
:100C0000DF6E12003901A3A7110093A711006F0036
:100C1000A0F757F03D01F9AB07D0F99B00019C4BC1
:100C20009D2B6F00A0F757F03D01F9A706D00001FA
:100C30009C4B9D2B6F00A0F757F0000E3724D96E08
:100C4000010E3820DA6E60005FF1DFFF010E3B26F7
:100C5000000E3C223D223E22010E3726000E382295
:100C600039223A224D50D8A420D03A5039103810A9
:100C700004E1400E375CD8A01100BC8A390193977B
:100C8000010E516E000E376E000E386E000E396E7A
:100C9000000E3A6E000E3B6E000E3C6E000E3D6E76
:100CA000000E3E6E010E4D6E11003A503910381094
:100CB0001AE1800E375CD8B016D0C00E5824016EF1
:100CC000FF0E5920026EFF0E5A20036EFF0E5B20AE
:100CD000046E3B50015C3C5002583D5003583E505E
:100CE0000458D8B01100BC8A39019397010E516E97
:100CF000110011C005F012C006F0030E086EE80ED8
:100D0000076E4FEC09F00550300F60004FF0D9FF2F
:100D1000600053F0DAFFDF6E20EE01F01350D926A9
:100D20001450DA22000E086E640E076E11C005F032
:100D300012C006F04FEC09F005C00CF006C00DF033
:100D4000000E0F6E0A0E0E6EE5EC09F00C50300F1F
:100D5000DF6E20EE02F01350D9261450DA22000E76
:100D6000086E0A0E076E11C005F012C006F04FECB7
:100D700009F005C00CF006C00DF0000E0F6E0A0E53
:100D80000E6EE5EC09F00C50300FDF6E20EE03F034
:100D90001350D9261450DA2211C00CF012C00DF0F5
:100DA000000E0F6E0A0E0E6EE5EC09F00C50300FBF
:100DB000DF6E20EE04F01350D9261450DA22000E14
:100DC000DF6E1200800E09140F6EFF0E0A14106EF3
:100DD000010E0B14116E000E0C14126ED2500F5037
:100DE00009180AE110500A1807E111500B1804E124
:100DF00012500C18D8B402D0FF0E120009C005F032
:100E00000AC006F00BC007F00CC008F05FEC0AF057
:100E100060002FF0F8FF60002BF0F7FF600027F074
:100E2000F6FF000E136E13500D24D96E000E0E2027
:100E3000DA6EDF50F56E7F0E1318D8A402D00C00C6
:100E400001D00D00132A7F0E1364EDD73901E5514F
:100E50003F0B8009E56FE585D29E3901E585550E8A
:100E6000E66FAA0EE66FE58300F0D28E00F0E595FE
:100E7000000E120034D011C009F012C00AF013C0E5
:100E80000BF014C00CF013C005F014C006F07AEC9F
:100E90000AF005C00DF006C00EF081EC07F0095015
:100EA0000A10D8A405D011C011F012C012F012001F
:100EB000010E1124056E000E1220066E60004FF028
:100EC000D9FF600053F0DAFFDF50156E1550076E42
:100ED000086A06EC0AF005C011F006C012F01150C5
:100EE0001210D8B409D0600047F0D9FF60004BF071
:100EF000DAFFDF50D8A4BFD7000E116E000E126EBD
:100F0000120034D0600027F0D9FF60002BF0DAFF28
:100F1000DF50D8B410D060002FF0D9FF600033F05C
:100F2000DAFF600027F0E1FF60002BF0E2FFDE5007
:100F3000E618D8B417D0600027F0D9FF60002BF076
:100F4000DAFFDF500F6E60002FF0D9FF600033F042
:100F5000DAFFDF50106E10500F5C096E0A6AD8A0DD
:100F60000A061200094A0A2A0B4A0C2A0D06D8A0C2
:100F70000E060D28C7E10E28D8A4C4D7000E0A6EAD
:100F8000000E096E12003901A3B76F00A0F757F0E9
:100F9000BC8A000E376E000E386E000E396E000EE1
:100FA0003A6E3A503910381013E1810E375CD8B0E0
:100FB0000FD0000E3724D96E010E3820DA6E000EE5
:100FC000DF6E010E3726000E382239223A22E9D789
:100FD0003901938D3D01F289000EF96F000EFA6F11
:100FE000000E576E000E0101006F000E516E000ED4
:100FF000376E000E386E000E396E000E3A6E000E1F
:10100000576EBC9A390193871200000EBA6E430ED8
:10101000C26E000E3A01406F000E416F000E426F2B
:1010200043694469BA96000EBB6ECF0EC36E000EC4
:10103000506F000E086F000E096F000E0A6F000E51
:101040000B6F080EC06F030E516F000E526F536985
:101050005469000EBC6E890EC46E000E606F000EE7
:10106000106F090E116F000E126F000E136F000E3D
:10107000146F000E156F130E166F170EE56FBC8AF6
:10108000000E626F0F0E636F646961691200000EDB
:101090000D6E000E0E6E000E0F6E000E106E0950DB
:1010A0000A100B100C10D8B42AD0010E116E06D005
:1010B000D89009360A360B360C36112A0CAEF8D702
:1010C000D8900D360E360F3610360950055C0A5092
:1010D00006580B5007580C500858D8A009D0095092
:1010E000055E0A50065A0B50075A0C50085A0D80DC
:1010F000D8900C320B320A320932112EE1D70DC0D2
:1011000005F00EC006F00FC007F010C008F0120086
:1011100005C00BF006C00CF019D00906D8A00A06CD
:1011200060001FF0D9FF600023F0DAFF074A082AA9
:1011300060002FF0E1FF600033F0E2FF0B4A0C2A61
:101140006F007FFFE7FFE750D8B40FD009500A10B7
:10115000D8B40BD0E2D760002FF0D9FF600033F095
:10116000DAFF000EDF6E0B4A0C2A0906D8A00A0629
:101170000928F1E10A28D8B41200EDD7165017104B
:1011800018101910D8B424D0010E1A6E06D0D890B9
:1011900016361736183619361A2A19AEF8D71650D9
:1011A000125C175013581850145819501558D8A0DD
:1011B00008D01650125E1750135A1850145A19506E
:1011C000155AD89019321832173216321A2EE7D71C
:1011D00012C012F013C013F014C014F015C015F0B3
:1011E0001200000E106E070E116E1150040DF35018
:1011F00007C00BF008C00CF009C00DF00AC00EF0DB
:10120000E82A05D0D8900E320D320C320B32E82E7F
:10121000F9D70B50126E12500F0B126E0A0E12609D
:1012200003D01250300F02D01250370F0F6E0F0E36
:10123000056E000E066E9EEC09F0110611BE12003E
:10124000D4D760001FF0F6FF600023F0F7FF08001E
:101250006F00D4FF49F017D060001FF0F6FF600068
:1012600023F0F7FF08006F00D4FF49F0600017F08B
:10127000D9FF60001BF0DAFF600027F1DFFF054AAD
:10128000062A074A082A4950D8A4E6D7600017F072
:10129000D9FF60001BF0DAFF000EDF6E1200000EB7
:1012A0000A6E000E096E07500810D8B41CD0010E4B
:1012B0000B6E04D0D890073608360B2A08AEFAD742
:1012C000D89009360A360750055C08500658D8A051
:1012D00005D00750055E0850065A0980D89008329C
:1012E00007320B2EEDD709C005F00AC006F0120038
:1012F000000E3D01EC6F000EED6F000EEE6F000E64
:10130000EF6F000EF06F000EF16FB00EF26F800EF7
:10131000F36F000EF46F8A0EF56F000EF66F000E7D
:10132000F76F000EF86F000EF96F000EFA6FF28B78
:10133000F289800EF46F390193971200000E406E0F
:10134000000E3F6E14D03901A3A9FDD73F500524EC
:10135000D96E40500620DA6EDF503D01EA6F3F4AF9
:10136000402A40500EE1810E3F5CD8B012003F5041
:101370000524D96E40500620DA6EDF50D8B4120032
:10138000E2D7120000EE00F2800EEE6AE806FDE100
:1013900000EE00F1820EEE6AE806FDE100EE60F07C
:1013A000980EEE6AE806FDE100EE2FF02D0EEE6AD3
:1013B000E806FDE1080ED56E000ED66E000ED76E63
:1013C000000EF86E000159EF00F00E500F10D8B467
:1013D00018D0010E106E04D0D8900E360F36102A99
:1013E0000FAEFAD70E500C5C0F500D58D8A004D099
:1013F0000E500C5E0F500D5AD8900F320E32102E38
:10140000F1D70CC00CF00DC00DF01200600017F009
:10141000D9FF60001BF0DAFF0750DE18D8A405D012
:1014200005C005F006C006F01200600017F0D9FFF5
:1014300060001BF0DAFF054A062ADF50D8A4E6D781
:10144000000E056E000E066E1200D28A000ED2BE8D
:10145000010E056ED29E550ED46EAA0ED46ED49097
:10146000000ED76E000ED66E080ED56E550ED46ED9
:10147000AA0ED46ED48005A002D0D28E01D0D29E06
:101480003901838712000FD03901A3A9FDD760006D
:1014900017F0F6FF60001BF0F7FF08006F00D7FFA2
:1014A000EAFD054A062A600017F0F6FF60001BF00F
:1014B000F7FF0800F5500009D8B41200E5D7D25064
:1014C00060001FF0F8FF60001BF0F7FF600017F0EE
:1014D000F6FF3901E5513F0B8009E56FE585E589A8
:1014E000D29E3901E585550EE66FAA0EE66FE583BB
:1014F000D28E120005C007F006C008F002D0074ADD
:10150000082A60001FF0D9FF600023F0DAFFDF50E7
:10151000D8A4F5D70550075C056E06500858066E2E
:101520001200000EAC6EAC508F0B3009AC6EF00E9A
:10153000AC16B40EAB6E000EAA6E010EAE6E040EAB
:10154000AF6E39019495A495AC8E12003901E55126
:101550003F0B8009E56F60001FF0F8FF60001BF093
:10156000F7FF600017F0F6FF0800F5501200000EBC
:101570007E6E7E987E867E847E927E903F015E9314
:101580005E81000E7F6E7E8E12003901A3A9FDD709
:101590000D0E3D01EA6F3901A3A9FDD70A0E3D01E9
:1015A000EA6F1200056E3901A3A9FDD7600017F09C
:1015B000EAFD1200FF00FF00FF00FF00FF00FF0038
:1015C000FF00FF00FF00FF00FF00FF00FF00FF0023
:1015D000FF00FF00FF00FF00FF00FF00FF00FF0013
:1015E000FF00FF00FF00FF00FF00FF00FF00FF0003
:1015F000FF00FF00FF00FF00FF00FF00FF00FF00F3
:10208000FF00FF00FF00FF00FF0000010000000A4A
:1020900000000064000000E803000010270000A01A
:1020A00086010040420F008096980000E1F505008F
:1020B000CA9A3B46696E20746573742073617469B3
:1020C0006E61730D0A002054657374205361746946
:1020D0006E61730D0A2045637269747572652034F0
:1020E0002064616E73206C61207A6F6E65203238D7
:1020F0003030682E2E3031464646462066616C737D
:10210000680D0A002050726F6A6574204D504C4172
:102110004258203A31384632374B34325F54657377
:10212000745F4563725F4C65635F466C6173685FA3
:10213000323032322D30392E580D0A00204574616C
:10214000706520300D0A2E2E20417474656E746502
:1021500020706F7572206361707475726520666996
:10216000636869657220776176200D0A00204A6FE6
:102170007565206C652066696368696572207761A2
:1021800076652073746F636BE920656E20666C6101
:1021900073680D0A00205461696C6C652044617499
:1021A00061203D20256C75206279746573200D0ACD
:1021B000204D6178426C6F633D20000D0A202D2D6B
:1021C0002D2D2D7265626F6F742064616E732032E5
:1021D000736563202D2D2D2D200D0A002041726D79
:1021E000652049565420696E7465727275707473F7
:1021F000202031384632374B34320D0A0020204738
:102200006C6F62616C2046696C652073697A652029
:102210003D20256C752062797465730D0A000D0AE6
:102220004365206E276573742070617320756E207E
:10223000574156202121212E2E2E0D0A000D0A2055
:1022400046696E206465206C6563747572652064F0
:1022500061746120776176650D0A00546F6F2042CA
:102260006967205761762066696C652064617461D6
:10227000732E2E0D0A0020457461706533202C6C7E
:102280006563747572652064617461730D0A00463C
:10229000696E207465737420736174696E61732054
:1022A0002E2E4F4B0D0A0020426C6F6323202020FE
:1022B0004C3220616472657373650D0A0020476CAF
:1022C0006F62616C2046696C652073697A65203D98
:1022D0002000457461706520310D0A205265E77554
:1022E000203A0D0A002045746170652034200D0AE3
:1022F0000057415645666D7420005249464600001D
:020000040020DA
:10000000FF0FFF0FFF0FFF0FFF0FFF0FFF0FFF0F80
:020000040030CA
:0A0000008CFFEFF79FFFFFFFFFFFEB
:00000001FF
